:020000040000FA
:02000000412B92
:08000800A000030EA10064003A
:100010001630810056206F20EC20210E8300A00EA8
:10002000200E0B110900FF30A800B630AB002530C0
:10003000AE002030B000B101B201B301B401B5018E
:10004000B601CA01CB01CC01CD01CE01CF01D00157
:10005000D101D201D3012511A5112513A601A616A0
:10006000F9210130D900DA000930DD000D30E0005F
:100070000330DE000800850107309F00031383165C
:10008000003085004030860003138312AC01AD01BF
:1000900008000B118B178B16810164000313831664
:1000A000D83081000313831281010800A51D6E283A
:1000B000251D6E28DB0B68288030DB00DA0B6828F2
:1000C0001030A506590859075907DA00DA03DA0390
:1000D000251E6E282D08803AAD0086000800A90A6A
:1000E0000319A80F7E28A514EF30A800FE30A90040
:1000F000AA0B7E28BC30A9002B08AA000800DE0845
:100100000319DF2837083102031D9A283808320204
:10011000031D9A2839083302031D9A283A0834022D
:10012000031D9A283B083502031D9A283C08360215
:100130000319B7283708BD003108B7003808BE00DA
:100140003208B8003908BF003308B9003A08C000C7
:100150003408BA003B08C1003508BB003C08C200A7
:100160003608BC006008E100E2005E08DF00E20B38
:10017000C1286008E200DF0BC1285E08DF00610BC8
:10018000E10061086202031CD2283708C300380866
:10019000C4003908C5003A08C6003B08C7003C083F
:1001A000C800EB283D08C3003E08C4003F08C50056
:1001B0004008C6004108C7004208C800EB283108C3
:1001C000C3003208C4003308C5003408C60035082F
:1001D000C7003608C80008002D088039AD00860029
:1001E000063032210830A2000310300C03182030F2
:1001F000B00030184308B018440830194508B01949
:100200004608301A4708B01A4808A202831C033E69
:10021000AC0085002D0880393004AD00A2002F0805
:100220003005031916292D088039AD00AE0B2D2994
:100230002530AE002208860000000608A2002D0826
:100240008600220840390319292922083F39D7049A
:100250002D292208FF3A3F39D7052D088600B01A0C
:100260007F200800A200A20B332908005708580677
:1002700003194B29A7015705D800D8194C21D818C4
:100280005621581A63215819702158187D21D81AFF
:100290008A215708D80008000310A60C0318522919
:1002A000F9215529A601A616F9210800A61A9721B9
:1002B000261A9E21A619A0212619DC21A618E321C1
:1002C0002618F8210800A61AC521261AB321A61956
:1002D000B5212619DE21A618EC212618F8210800E0
:1002E000A61AC821261ACF21A619CF212619CF2157
:1002F000A618CF212618F8210800A61AC521261A0B
:10030000D021A619D8212619E021A618BE21261829
:10031000F8210800A61AC521261AD321A619D3212F
:100320002619D321A618D3212618D3210800251178
:100330000830A5061030B606A512080015230800DF
:1003400052082923D200251CA82953083523D3009D
:100350005308023C031DB2295208043C031DB22974
:10036000D201D30108000B23080050082923D00034
:10037000251CBD2951083523D1000800DE0A5E087E
:10038000093C03180800DE010800A5122511080029
:10039000251DCE292511A5165D08DC0008000800E2
:1003A000CA01CB0108002511A601A616F9210800F3
:1003B0005D082923DD000800AB030800AB0A080034
:1003C0004030A5060800A5151030B6042515D90B38
:1003D000EB290930D9000800A5151030B604251501
:1003E000D90A5908093C0318F729D901D90A080084
:1003F0000800EF30B105B205B305B405B5051030FE
:10040000261AB504A619B4042619B304A618B20412
:100410002618B1040800A61A1822261A1822A619AE
:10042000592226197322A618A7222618BE220800D0
:100430003108F0394A04B1003208F0394B04B200F7
:100440003308F0394C04B3003408F0394D04B400DB
:100450004E08A3004F08A400A61E492A251F492ABA
:10046000CF080319432ACF18392A4E08023C031833
:10047000492AA303A303A31F412A23080A3EA3007A
:10048000A403A403492ACE08031D492AA30AA30AE8
:10049000A40A3508F0392304B5003608F0392404DD
:1004A000B600B608031D572A2030AF00582AAF0106
:1004B00008000230AF003108F0395D04B1003208A5
:1004C000F039B2003308F0395004B3003408F03981
:1004D0005104B4003508F0395204B5003608F0393B
:1004E0005304B60008000830AF00D501D6012B0830
:1004F000D4006430D60AD40203187A2AD407D6036B
:100500000A30D50AD4020318812AD407D50331084A
:10051000F0395404B1003208F0395504B200330800
:10052000F0395604B3003408F039B4000230251F06
:100530000430A3003508F0392304B5000130251F2D
:100540000230A3003608F0392304B6000800243036
:10055000AF003108F0395904B1003208F039B20067
:100560003308F039B3003408F0395E04B4003508BC
:10057000F039B5003608F039B6000800AF0131088F
:10058000F039B1003208F039B2003308F039B30065
:100590003408F039B4003508F039B5003608F039C0
:1005A000B6000800CA08031DEB2ACB08031DEB2A7E
:1005B0004C085002031DEA2A4D085102031DEA2A85
:1005C0004E085202031DEA2A4F085302031DEA2A6D
:1005D0002515EB2A25110800A51EF22ADC0BF22AAC
:1005E0002515A5120800A70A14302702031CFB2AB0
:1005F000A601A616F9210800A51C282BA510F32298
:100600004A082923CA00251C272B4B083523CB0079
:10061000251C272BEC224C082923CC00251C272B3A
:100620004D083523CD00251C272B4E082923CE004D
:10063000251C1D2B4F082923CF004F08023C031D0A
:10064000272B4E08043C031D272BCE01CF01D222BD
:1006500008002510C900490AC900093C0318332BBA
:1006600000302514342B490808002510C900490A18
:10067000C900053C03183F2B00302514402B4908C6
:10068000080013203B2049203621FC220B22442B5A
:02400E00053F6C
:00000001FF
